S01B00006275696C642F6D69636132646F742F6D61696E2E73726563E3
S11300000C945F010C947C010C947C010C947C0195
S11300100C947C010C947C010C947C010C947C0168
S11300200C947C010C947C010C947C010C947C0158
S11300300C947C010C947C010C947C010C94C20BF8
S11300400C947C010C947E010C9406020C947C01AB
S11300500C9430020C9409080C947C010C947C01DF
S11300600C947C010C947C010C947C010C947C0118
S11300700C947C010C947C010C947C010C947C0108
S11300800C947C010C947C010C947C01001C005E9B
S113009000FA017301EA04BC0A5E050202020202CC
S11300A002000000140055008700B901E5043D007A
S11300B0080808080808AEEFEFEFEFEFEF000021A3
S11300C010422063308440A550C660E7700881293F
S11300D0914AA16BB18CC1ADD1CEE1EFF1311210D7
S11300E00273325222B5529442F772D6623993188F
S11300F0837BB35AA3BDD39CC3FFF3DEE3622443E3
S11301003420040114E664C774A44485546AA54BDE
S1130110B528850995EEE5CFF5ACC58DD553367276
S11301202611163006D776F6669556B4465BB77A2E
S1130130A719973887DFF7FEE79DD7BCC7C448E502
S1130140588668A7784008611802282338CCC9ED7E
S1130150D98EE9AFF9488969990AA92BB9F55AD416
S11301604AB77A966A711A500A333A122AFDDBDCCE
S1130170CBBFFB9EEB799B588B3BBB1AABA66C8722
S11301807CE44CC55C222C033C600C411CAEED8F1E
S1130190FDECCDCDDD2AAD0BBD688D499D977EB6B6
S11301A06ED55EF44E133E322E511E700E9FFFBE6E
S11301B0EFDDDFFCCF1BBF3AAF599F788F8891A941
S11301C081CAB1EBA10CD12DC14EF16FE18010A118
S11301D000C230E3200450254046706760B983981C
S11301E093FBA3DAB33DC31CD37FE35EF3B1029068
S11301F012F322D2323542145277625672EAB5CBE8
S1130200A5A89589856EF54FE52CD50DC5E234C3B7
S113021024A01481046674476424540544DBA7FABB
S1130220B79987B8975FE77EF71DC73CD7D326F207
S1130230369106B01657667676154634564CD96D07
S1130240C90EF92FE9C899E9898AB9ABA944586557
S11302504806782768C018E1088238A3287DCB5C5B
S1130260DB3FEB1EFBF98BD89BBBAB9ABB754A54A7
S11302705A376A167AF10AD01AB32A923A2EFD0F27
S1130280ED6CDD4DCDAABD8BADE89DC98D267C07F7
S11302906C645C454CA23C832CE01CC10C1FEF3EFB
S11302A0FF5DCF7CDF9BAFBABFD98FF89F176E3647
S11302B07E554E745E932EB23ED10EF01E00112474
S11302C01FBECFEFD0E1DEBFCDBF11E0A0E0B1E0B3
S11302D0E6E3FDE200E00BBF02C007900D92AC34F0
S11302E0B107D9F712E0ACE4B1E001C01D92A23D20
S11302F0B107E1F70C947D020C9400001F920F9259
S11303000FB60F9211242F933F934F935F936F93E4
S11303107F938F939F93AF93BF93EF93FF939FB17B
S1130320809108028FB9892F0E94CA08FF91EF912A
S1130330BF91AF919F918F917F916F915F914F91F9
S11303403F912F910F900FBE0F901F901895AF9271
S1130350BF92CF92DF92EF92FF920F931F93CF93AE
S1130360DF9386EEF82EA090C102B090C202C09036
S1130370C302D090C402A114B104C104D10481F118
S1130380EE246FE572E000E010E081E090E0002EE2
S113039002C0880F991F0A94E2F7AA2797FDA09537
S11303A0BA2F8A219B21AC21BD210097A105B1055B
S11303B079F02F2D332744275527FB01858196811A
S11303C0A781B08582179307A407B5070CF4F580BD
S11303D0E3940F5F1F4F675F7F4FF2E0FE15A8F6AF
S11303E08FB7F8949927F0928E02F1BE109283028F
S11303F08FBF0E94B007DF91CF911F910F91FF90A3
S1130400EF90DF90CF90BF90AF9008951F920F921E
S11304100FB60F9211242F933F934F935F936F93D3
S11304207F938F939F93AF93BF93EF93FF935F9BC0
S113043006C08CB140E050E060E00E94AC0CFF913B
S1130440EF91BF91AF919F918F917F916F915F9148
S11304504F913F912F910F900FBE0F901F901895C1
S113046078941F920F920FB60F9211242F933F93FB
S11304704F935F936F937F938F939F93AF93BF93A8
S1130480EF93FF930E94780EFF91EF91BF91AF918C
S11304909F918F917F916F915F914F913F912F9198
S11304A00F900FBE0F901F901895AC018FB7F89462
S11304B0282F3327E0918002809180028F5F809300
S11304C080028091800287708093800290918002E4
S11304D080912A02981759F02FBFFF27EE0FFF1FB4
S11304E0EF50FE4F4083518381E090E00895E09304
S11304F080022FBF80E090E00895C5EED0E1DEBF1A
S1130500CDBF1ABA17BA11BA92E092B993B9D29A76
S1130510D09AD19A8B98809161008F7780936100F3
S11305201798A79AA69AA59AA49AA39AA29AA19A66
S1130530A09A8D9A8F9A8E9ABB98BF98159AD79A3B
S1130540D39A1D9ADF9ADA9A9F5F9C5F9739E8F3F2
S113055010E08AE08093E0011093800210932A0255
S11305601093D1028FB7F894992710937A028FBF12
S11305708FB7F89499271093A302DA9AD89AD99A44
S11305808FBF812F8B5F8093C50181E08093C6016B
S11305900E945E061093B401DB98D39ADF9AD79A2F
S11305A0DE98D6980E945E060E948D068FB7F89456
S11305B09927109385028FBFB1E0EB2EF12C8FB7F2
S11305C0F894282F3327E092B101812F8E5F809316
S11305D04C018FE292E09093820280938102109307
S11305E0330282E290E090937C0280937B0210932A
S11305F0EE011092CA021092C9021092E9011092FF
S1130600E80110920302109202021093AF011093BA
S1130610A90110939E028FEF9FEF9093870280931E
S11306208602909389028093880210935E0210934D
S11306308C02E6EBF0E08491992790935B0280931F
S11306405A022FBF8FB7F8949927B998BB98BA98D4
S11306506B986A986F9A6E9A8FBF17988D9A8E9A34
S11306608F9A959A979A969A6AE3812F0E94D10657
S11306706BE3812F0E94D10680ED97E00197F1F79B
S113068080E880931402682F8BE00E94D10680E9F1
S113069080931602682F8C580E94D106109318027A
S11306A08FE68093190285E580931A02612F8FE00B
S11306B00E94D10680911902682F80E10E94D10620
S11306C080911A02682F81E10E94D106E0921C02F7
S11306D06E2D83E10E94D106E092270219821A82CC
S11306E01B821C8220E030E040E050E02D833E83FA
S11306F04F835887BA01A90149875A876B877C873A
S11307006FEF7FEF8FEF9FE76D877E878F87988BE3
S1130710198A1A8A1B8B1C8B83E091E08D8B9E8B2C
S1130720A7E2B1E0AF8BB88FE0E0F0E0E98FFA8F99
S1130730AD89BE89AD90BD90CD90DD90AD8BBE8B63
S1130740EE24FF2487011701280160E070E885E4A6
S113075097E6A60195010E947916DA01C901817014
S11307609070A070B070892B21F02F5F3F4F4F4FD6
S11307705F4F21FF0BC0212CA0E23A2E412C512CBB
S11307808601750116950795F794E794E2E056956E
S1130790479537952795EA95D1F7DA01C9017EE0A7
S11307A0880F991FAA1FBB1F7A95D1F7820D931D3D
S11307B0A41DB51D212C60EE362E6FEF462E6FEF73
S11307C0562E280E391E4A1E5B1E80509042A044AD
S11307D0B04080509C49AF4BB04008F060C0AF8936
S11307E0B88D8D919C91AA27BB2742013101681ACB
S11307F0790A8A0A9B0AD401C30180509040A0441C
S1130800B04080509C49AF4BB04008F048C0CA018A
S1130810B901A60195010E945A16DC01CB01E80E2C
S1130820F91E0A1F1B1F20E136EB4DEF5FEFE20EAE
S1130830F31E041F151FD801C70180519641AF4C08
S1130840B941B7FF07C0B095A095909581959F4F8A
S1130850AF4FBF4F4D855E856F85788984179507A7
S1130860A607B707E4F42D823E824F825886698634
S11308707A868B869C86E982FA820B831C83298D77
S11308803A8D275C3E4FF90120813181298B3A8BC7
S1130890FC89FA5FFB8B8D879E87AF87B88B2C8989
S11308A02F5F2C8B498D5A8D4E5F5F4F498F5A8F26
S11308B06F89788D6E5F7F4F6F8B788F293008F446
S11308C037CF7B89772309F460C08D8180930C0234
S11308D02D813E814F815885BB27A52F942F832FCF
S11308E080930B02CA01AA27BB2780930A02398589
S11308F030930F0249855A856B857C85BB27A72FCA
S1130900962F852F80930E02CB01AA27BB278093B5
S11309100D0259895093110269897A89872F992781
S11309208093100289819A81AB81BC818030E5E695
S11309309E07EDECAE07EDE1BE07A8F480509448A5
S1130940A74DB74128F484E88093120281E904C0DA
S113095084E48093120281E88093260282E08093EB
S1130960130280E70AC08CE88093120283EF80931D
S1130970260282E38093130280E280931B022B8978
S1130980220F220F220F2093150249815A816B8175
S11309907C814093C5025093C6026093C702709352
S11309A0C80211E06AE0E62E62E0F62ED7018D91CE
S11309B07D01682F812F0E94D1061F5F1D30B0F387
S11309C080911B02682F82E10E94D10660E08BE0D7
S11309D00E94D1066FE382E40E94D10661E180E0C7
S11309E00E94D10666EA8EE00E94D1068EE00E9443
S11309F0F50683FFFBCF66E28EE00E94D10661EE2E
S1130A0080E00E94D10680912602682F89E00E942E
S1130A10D10660E08BE00E94D10666EA8EE00E9477
S1130A20D1061EE0812F0E94F50683FFFACF66E20D
S1130A30812F0E94D10680E980931602682F8DE0F1
S1130A400E94D10680912702282F33278FB7F8946C
S1130A5099272093B6028FBF0E9428078FB7F89476
S1130A6099271092A8028FBF8FB7F89499271092F4
S1130A70D0021092CF021092A7021092A6021092F6
S1130A802E0210922D028FBF0E9428078FB7F89470
S1130A90992716B917B88FBF8FB7F894482F5527E1
S1130AA0209100013091010181E597E3289FF00135
S1130AB0299FF00D389FF00D1124CF018F5A984CC7
S1130AC090939C0280939B029093CD028093CC02DE
S1130AD085E89FE0289FB001299F700D389F700D15
S1130AE01124CB018B57904F9093E2018093E10145
S1130AF04FBF0E945E068091000190910101909386
S1130B00BE028093BD021092C0021092BB021092EA
S1130B10BA0210925D0210925C028091B4018823A3
S1130B2069F481E08093B4018AEB91E09093AB0186
S1130B308093AA0186EF90E10E9455020E948D06DF
S1130B40109290008CE089B98CB11BB8A6E0A093F8
S1130B50950088ED8AB98FB7F89499276091B1010F
S1130B608FBF613009F06CC08FB7F894482F5527B8
S1130B70E0918102F0918202148272E07093B101DB
S1130B801092A9011092AF018FEF9FEF909387020B
S1130B908093860280915E029927880F991FFC0139
S1130BA0E457FF4F24913327322F222783579F4F37
S1130BB0FC0184919927282B392B3093E70120934A
S1130BC0E6014FBF10918C021123D1F46BE3812F06
S1130BD00E94D10680ED97E00197F1F769E3812F38
S1130BE00E94D10688EC90E00197F1F7BB98BA987F
S1130BF00E94C20780EC8DB9B8980E94B00720C04B
S1130C00812F9927880F991FFC01EF55FF4F2491DD
S1130C103327322F22278E559F4FFC018491992729
S1130C20282B392B8FB7F8949927A093B1018FBF44
S1130C30C901AA27BB279C01AD01872F0E94430746
S1130C4028EE33E040E050E060E081E00E9443079A
S1130C501092C0020E94B007789490912A02809169
S1130C608002981719F480E090E01FC08FB7F894C1
S1130C70282F332790912A0280912A028F5F809334
S1130C802A0280912A02877080932A02E92FFF2783
S1130C90EE0FFF1FEF50FE4F808191811082118271
S1130CA02FBFFC01099581E090E08823B1F685B758
S1130CB0806285BF889500000000CFCF1092C102EA
S1130CC01092C2021092C3021092C40210928302C4
S1130CD08FEF8093CB028093A7011092EF0183E002
S1130CE08093840296EE90938E028FB7F894282F07
S1130CF0332787B78E7F87BF87B78D7F87BF80B73E
S1130D00886080BF8BE083BF12BE91BF87B78260CB
S1130D1087BF2FBF81E090E008958FB7F894682FC4
S1130D2080E090E04FE451E09C01F901E80FF91FE5
S1130D30E157FD4F44835583128213821182019639
S1130D402B5F3F4F455D5F4F8230910574F31092E6
S1130D50B50210927E0210927D021092B30110929D
S1130D60B20110924E0110924D011092A601109200
S1130D70A5011092B40210928A021092B702109246
S1130D80E5011092E4011092050210920402809190
S1130D909302909194029093A1028093A0026FBF5A
S1130DA00895880F959896E087FF02C0979A01C02E
S1130DB097989698969A880F915097FFF5CF979A9F
S1130DC09698969A959A97E067FF02C0979A01C001
S1130DD097989698969A660F915097FFF5CF959AA3
S1130DE0979A969A81E090E0089590E0880F9598FC
S1130DF026E030E087FF02C0979A01C09798969842
S1130E00969A880F2150304037FFF4CF27E030E026
S1130E1097989698969A8F98959A969840E050E06D
S1130E20879941E0892F992721503040442329F0A4
S1130E30880F991F982F916002C0982F990F969A46
S1130E4037FFEBCF959A8F9A979A892F9927089510
S1130E508FB7F894282F8091E301882391F480E0E0
S1130E6090E0E8EAF2E0819301968C309105DCF39E
S1130E708EE18093B2028FE18093B30281E080938C
S1130E80E3012FBF0895CF92DF92EF92FF920F9369
S1130E901F93CF93DF9379018A01833010F462307A
S1130EA01CF080E090E053C0282F3327F90173E051
S1130EB0EE0FFF1F7A95E1F7E20FF31FE15AFD4FA2
S1130EC0E182F2820383148360838FB7F894C82F7E
S1130ED0DD2782B7E80EF11C011D111DE582F682A3
S1130EE00783108751E0C52ED12CC60102C0880F9C
S1130EF0991F2A95E2F79C01442737FD4095542F0A
S1130F008091C1029091C202A091C302B091C40227
S1130F10822B932BA42BB52B8093C1029093C202F6
S1130F20A093C302B093C40280918E029927AA278A
S1130F30BB27E816F9060A071B0738F4E0928E026D
S1130F40E1BE109283020E94B007CFBFC601DF91B9
S1130F50CF911F910F91FF90EF90DF90CF90089564
S1130F6080914B01882329F48CE490E10E9455027E
S1130F7006C085B7837E85BF85B7806285BF80E064
S1130F8090E008951F9310E061E1812F0E94D10643
S1130F9080911202682F89E00E94D106612F8BE0B4
S1130FA00E94D1068AEF90E00197F1F781E090E08A
S1130FB01F910895FC01209100013091010180915D
S1130FC05C0290915D02019690935D0280935C02B5
S1130FD082A193A10197D9F493818091020198177A
S1130FE0B1F4808191814FEF8F3F940719F08217FC
S1130FF0930769F4928183E08C5F8B32E8F390323B
S113100031F4858196819093C8018093C701CF0103
S113101008951F920F920FB60F921124FF920F930F
S11310201F932F933F934F935F936F937F938F936C
S11310309F93AF93BF93CF93DF93EF93FF93C4B189
S1131040D5B1D370349A379878948FB7F894F82E32
S11310508091CF02082F112721E030E0002E02C03A
S1131060220F331F0A94E2F78091A6029091A702FF
S113107082239323892B61F42095309580912D024E
S113108090912E028223932390932E0280932D021B
S113109040912D0250912E024115510511F12091DC
S11310A0CF023091D0022F5F3F4F2C30310511F029
S11310B0C90102C080E090E09C0181E090E0022E32
S11310C002C0880F991F0A94E2F784239523892B81
S11310D051F33093D0022093CF028091CF020E942B
S11310E0B808FFBE0115110569F48FB7F894282FCD
S11310F03327D0938902C093880281E080939E02B3
S11311002FBF01C080E099272FB7F8948823C9F432
S113111061E070E002C0660F771F0A95E2F7409124
S1131120A6025091A702CA0186239723892B49F06E
S1131130CB0180959095482359235093A70240935F
S1131140A6022FBFFF91EF91DF91CF91BF91AF9195
S11311509F918F917F916F915F914F913F912F91CB
S11311601F910F91FF900F900FBE0F901F90189535
S1131170982F8FB7F894282F3327E8EAF2E0E90F85
S1131180F11D80818F7187B92FBF379A369A81E01C
S113119090E008951F93CF93682F8091B602811138
S11311A060958091B101482F55274230510509F4CB
S11311B0ADC04330510524F44115510571F0A3C26B
S11311C04430510509F469C1443051050CF404C19B
S11311D04530510509F4D9C196C22091A2028FB7B6
S11311E0F8949927209308028FBF6091B8027091F8
S11311F0B9026F5F7F4F7093B9026093B802809118
S11312004C0199278430910559F18530910534F4C6
S11312108230910559F00397B1F06AC08630910588
S113122009F45EC006970CF44BC062C08091E601DD
S11312309091E7016817790708F465C283E3809306
S1131240A20283E052C08CEC8093A20284E08093DB
S11312504C018FEF9FEF9093B9028093B80253C271
S11312608091B802282F33278091EA019091EB01F5
S113127028173907F8F4E091A402F091A502E60FCB
S1131280F71F20812093A202809106029091070209
S1131290EDEBF0E02927220FF11DE20FF11DC895B7
S11312A0982F802D3196C8959025909307028093AE
S11312B0060229C2809106028093A20285E015C02D
S11312C08091060290910702892F99278093A202A8
S11312D086E080934C015093B9024093B80213C244
S11312E06430710508F40FC287E080934C010BC28F
S11312F0BB98BA980E94C2071092AF018AE89FE097
S11313000E945502882309F4FEC19AC16A3A11F079
S1131310653571F52091C9023091CA022F5F3F4FA4
S11313203093CA022093C90280918C02E82FFF27D0
S1131330E656FF4F849199278217930708F0E3C17B
S11313401092BF021092CA021092C90210922C028B
S113135010922B021092EE011092070210920602D4
S113136082E290E090937C0280937B0284E069C1E6
S11313708091AF01882309F4C6C1809186029091BF
S113138087020197909387028093860218161906A4
S11313900CF4B9C110929E028FB7F894C82F209113
S11313A02D0230912E0220FD10C0C901816090935E
S11313B02E0280932D022115310539F43093D00289
S11313C02093CF0280E00E94B808CFBF1092CA02D7
S11313D01092C90283E035C16A3A09F449C06535FF
S11313E009F446C080919E02882309F48CC180913F
S11313F08C02E82FFF27EA54FF4F8491282F3327CC
S113140080918802909189022817390788F561EE46
S113141080E00E94D10680912602682F89E00E9414
S1131420D1068AEF90E00197F1F780911402682FBA
S11314308BE00E94D10684E190E00197F1F7BB9A1A
S1131440BA9A1092B9021092B8021092070210923E
S113145006021092B10182E080934C012AEA2093A3
S1131460A2028FB7F8949927209308028FBF4BC12B
S11314700E94970B8F70907024E230E0829FA0014D
S1131480839F500D929F500D1124CA01820F931F08
S11314909093870280938602D3C06A3A11F065352F
S11314A019F4609303022FC18091BF02992700971A
S11314B021F003970CF060C003C0609302025FC088
S11314C02091020230910302922F88279093030205
S11314D0809302026093020210E0220F331F67FD23
S11314E02160660F53E32C3C350709F040C0E091BE
S11314F08102F091820244814423B9F08FB7F894B9
S1131500382F2091A30220FF06C08FB7F8949927A3
S1131510DA9A2E7F05C08FB7F8949927DA9821605C
S11315202093A3028FBF3FBF27C085E08093B10102
S11315308FB7F894C82F20912D0230912E0220FDF0
S113154010C0C901816090932E0280932D02211551
S1131550310539F43093D0022093CF02842F0E94B6
S1131560B808CFBF87E0811B8093EE0108C01F5FDE
S1131570183008F4B2CF03C082E08093B1018091A7
S1131580BF028F5F8093BF02BEC080910202909120
S11315900302982F8827909303028093020260939A
S11315A0020220910202309103020090EE0102C077
S11315B0369527950A94E2F7622FE0918102F09123
S11315C0820280912B0290912C02E80FF91F208354
S11315D040912B0250912C024F5F5F4F50932C028D
S11315E040932B0280917B0290917C02481759070B
S11315F098F58091060290910702EDEBF0E06927DF
S1131600660FF11DE60FF11DC895982F802D3196B8
S1131610C8959025909307028093060245305105A2
S113162009F071C0E0918102F091820284819927CE
S113163090937C0280937B028E31910528F0148272
S113164082E08093B1015FC00097F1F0059690931A
S11316507C0280937B0257C048175907E1F48091BC
S1131660060290910702EDEBF0E06927660FF11D89
S1131670E60FF11DC895982F802D3196C8959025B9
S1131680909307028093060282E290E090932C02EA
S113169080932B0238C044325105A8F1E0918102B5
S11316A0F091820222A133A1809106029091070257
S11316B02817390729F481E090E082A393A302C09C
S11316C012A213A20E94BA0BC2E0C093B101E0912E
S11316D08102F0918202809188029091890284A310
S11316E095A388E49FE00E945502882361F4E09169
S11316F08102F09182028483C093B10180EC8DB9A0
S1131700B8980E94B00781E090E0CF911F910895AE
S1131710FC011092C00282818A3031F48FB7F894B0
S1131720992710927A028FBF81E090E008958FB7D5
S1131730F894482F552720919B0230919C02832FC7
S1131740881F8827881F220F331F882321F08BE0EE
S113175090E1282739272F5F3F4F30939C02209335
S11317609B028091E1019091E201282739274FBF24
S1131770C90108956F98B89AC0980E94B00781E093
S113178090E0089578941F920F920FB60F9211244F
S11317902F933F934F935F936F937F938F939F9375
S11317A0AF93BF93EF93FF938FB7F894282F33270A
S11317B08091F001882369F080917F0280939F02D9
S11317C0886080937F0283BF8091010281BF109261
S11317D0F0012FBF8FE99FE00E945502FF91EF9126
S11317E0BF91AF919F918F917F916F915F914F9135
S11317F03F912F910F900FBE0F901F901895CF938C
S1131800C1E020E08FB7F894382F8091B502882387
S113181091F58091CE02992781FF08C08BE892E070
S1131820909329028093280280E41AC082FF0FC09B
S1131830E091A501F091A601F0932902E09328021A
S113184082E48093A8018481992705960DC083FFC3
S113185012C080EB91E090932902809328028FEFCD
S11318608093A80181E090E09093B3018093B2014A
S11318702C2FC093B5023FBF2223F1F08FB7F89409
S1131880992710924E0110924D0110927E021092EF
S11318907D028FBF8EE70E94600CC82F813061F0FB
S11318A08FB7F894282F332788E08093B5022FBF91
S11318B085E79CE00E9455028C2F9927CF910895CB
S11318C0482F8FB7F894282F33279091850281E011
S11318D0809385022FBF992319F080E090E008954A
S11318E04CB95E9A81E090E0089561E08FB7F89476
S11318F0282F33278091B502883019F460E0609373
S1131900B5022FBF8091A8019091CE02803451F48A
S11319108FB7F894282F332782E098279093CE022C
S11319202FBF17C08FB7F894282F332784E0982748
S11319309093CE022FBF8091A5019091A6010E94A1
S1131940880B8FB7F89499271092A6011092A501DD
S11319508FBF0E94FF0B0895382F8091B4029927FE
S11319608230910509F46BC0833091052CF4009703
S113197059F0019781F1B7C18330910509F49CC0F6
S1131980049709F459C1AFC13E3709F0AEC1809143
S11319908A029927FC01EE0FFF1FEE0FFF1FE80FCD
S11319A0F91FE80FF91FE157FD4F828193810097DA
S11319B009F09BC1118290930502809304029093D5
S11319C0E5018093E401848195819093A102809341
S11319D0A00281E085C13E3709F487C180918A0263
S11319E09927FC01EE0FFF1FEE0FFF1FE80FF91FF1
S11319F0E80FF91FE157FD4F308380910402909165
S1131A000502EDEBF0E0232F2927220FF11DE20F51
S1131A10F11DC895982F802D3196C89590259093E7
S1131A20050280930402832F99278134910529F0BC
S1131A308234910509F453C156C182E051C13E3745
S1131A4009F451C160918A023D3781F4862F9927A8
S1131A50FC01EE0FFF1FEE0FFF1FE80FF91FE80F49
S1131A60F91FE157FD4F80E281833FC1862F9927FB
S1131A70FC01EE0FFF1FEE0FFF1FE80FF91FE80F29
S1131A80F91FE157FD4F218123272183809104020F
S1131A9090910502EDEBF0E02927220FF11DE20FF2
S1131AA0F11DC895982F802D3196C8959025909357
S1131AB005028093040213C14091E4015091E501B1
S1131AC04C32510508F0BAC03D3711F484E008C126
S1131AD03E3709F07FC04230510508F45FC0E09101
S1131AE0A002F091A102E40FF51F82919927382FEB
S1131AF0222782919927282B392B809104029091D7
S1131B00050260918A0228173907E1F4862F992784
S1131B10FC01EE0FFF1FEE0FFF1FE80FF91FE80F88
S1131B20F91FE157FD4F425050404283538384E8EC
S1131B3090E10E94550280918A028F5F81708093A8
S1131B408A0210C0862F9927FC01EE0FFF1FEE0FAB
S1131B50FF1FE80FF91FE80FF91FE157FD4F12822D
S1131B601382118280918A029927FC01EE0FFF1FD4
S1131B70EE0FFF1FE80FF91FE80FF91FE157FD4FA4
S1131B8082819381892BD9F4848195819093A102D8
S1131B908093A00281E08093B40213C080918A02F2
S1131BA09927FC01EE0FFF1FEE0FFF1FE80FF91F2F
S1131BB0E80FF91FE157FD4F128213821182109230
S1131BC0B40210920502109204021092E5011092E0
S1131BD0E4018BC0E091A002F091A102E40FF51F93
S1131BE030834091E4015091E50142305105E8F021
S1131BF02091040230910502E091A002F091A1022B
S1131C00E40FF51F32978081EDEBF0E08327880F16
S1131C10F11DE80FF11DC895322F202D3196C8957E
S1131C20302530930502209304024F5F5F4F509399
S1131C30E5014093E40159C03E37D1F41092050206
S1131C40109204021092E5011092E40180918A023C
S1131C509927FC01EE0FFF1FEE0FFF1FE80FF91F7E
S1131C60E80FF91FE157FD4F1282138211823BC026
S1131C7080E28327E091A002F091A1022091E40187
S1131C803091E501E20FF31F80834091E40150910C
S1131C90E50142305105E8F020910402309105023B
S1131CA0E091A002F091A102E40FF51F3297808128
S1131CB0EDEBF0E08327880FF11DE80FF11DC895C7
S1131CC0322F202D3196C89530253093050220936C
S1131CD004024F5F5F4F5093E5014093E40183E0BA
S1131CE08093B40202C01092B40281E090E008959F
S1131CF08FB7F894992720918502109285028FBF9F
S1131D00222309F4A4C08091B502873031F41092E3
S1131D10B50285E79CE00E94550221E08091B5025E
S1131D2099278430910509F46EC08530910554F4E7
S1131D308230910561F1833091050CF058C0019710
S1131D4049F07CC08630910509F471C006970CF403
S1131D5063C074C082E08093B50220914D0130913C
S1131D604E018091A801EDEBF0E08327880FF11D6F
S1131D70E80FF11DC895322F202D3196C8953025D6
S1131D8030934E0120934D018091A80154C0E091FD
S1131D902802F091290220917D0230917E02E20F07
S1131DA0F31F508180914D0190914E01EDEBF0E0D5
S1131DB0452F4927440FF11DE40FF11DC895982FB5
S1131DC0802D3196C895902590934E0180934D01B6
S1131DD02F5F3F4F30937E0220937D028091B201AA
S1131DE09091B3012817390798F084E00FC08091CF
S1131DF0BC0290E289270E94600C282F80919D02EA
S1131E008093B5021BC050914D0185E08093B502CB
S1131E10852F0E942A0F11C080914D0190914E018F
S1131E20292F332786E08093B502822FF2CF87E0F3
S1131E308093B5028EE70E94600C282F213039F080
S1131E4088E08093B50285E79CE00E94550281E01A
S1131E5090E00895982F8D57823078F48FB7F894D6
S1131E60282F33278091B50280939D0283E08093CD
S1131E70B5029093BC022FBF9DE7892F0E94600C8E
S1131E80992708958FBF08958FB7F89499270895D7
S1131E908FB7F894682F7727E0918102F09182023E
S1131EA017A210A684A195A19C01220F331F220F13
S1131EB0331F280F391F40915A0250915B02CA0107
S1131EC0880F991F840F951F280F391F53E03695EB
S1131ED027955A95E1F730935B0220935A026FBF1E
S1131EE0CF010E94DA079C018FB7F8949927211536
S1131EF0310521F03093820220938102E091810226
S1131F00F091820214828FBF80EC8DB9B8980E9440
S1131F10B00708958FB7F8949927E091A402F0913F
S1131F20A50217A210A68FBF61E0CF010E94880B03
S1131F308FB7F89499271092A9018FBF08958F92B3
S1131F409F92AF92BF92DF92EF92FF920F931F93F3
S1131F50CF93DF9381E0809383028091C1029091BB
S1131F60C202A091C302B091C4020097A105B105B9
S1131F7009F484C0DD240FE512E0EE24FF2461E0BF
S1131F8070E00E2C02C0660F771F0A94E2F7CB01B3
S1131F90AA2797FDA095BA2F8090C1029090C20203
S1131FA0A090C302B090C40288219921AA21BB2128
S1131FB00097A105B10509F457C080918E029927B5
S1131FC00196AA2797FDA095BA2FF801258136819D
S1131FD047815085281B390B4A0B5B0B25833683BD
S1131FE0478350872330310541055105ECF5808145
S1131FF0882369F481819281A381B481280F391FD8
S11320004A1F5B1F258336834783508713C0CB0148
S113201080959095AA2797FDA095BA2F882299229A
S1132020AA22BB228092C1029092C202A092C30251
S1132030B092C4028091CB02823019F48FEF809366
S1132040CB029091CB029F5F9093CB028091EF01E2
S11320508F5F8093EF01E92FFF27E455FE4FD08275
S11320608DE794E10E945502D3940894E11CF11C7D
S1132070075F1F4FF2E0FD1508F081CF0E94A70112
S1132080DF91CF911F910F91FF90EF90DF90BF9060
S1132090AF909F908F90089587B799278C7F009772
S11320A019F080E090E01AC06F9918C0379B03C004
S11320B088E090E013C087B7992783709070892BCC
S11320C059F081B792B7891B803118F48CE190E004
S11320D005C088E190E002C080E190E0382F25B788
S11320E0237E8C3121F0883111F008C0000080B7C4
S11320F0992787709070892BC9F7237E232B25BFDE
S113210085B7806285BF08950F931F93CF93DF93A4
S11321109091B70286E0989F8001112401571D4FCA
S1132120F801C481D58182819381059780F1208152
S1132130822F99278134910559F08234910524F432
S11321408034910521F11DC08234910571F019C0CC
S113215081E090E08AA39BA3F801818180938D02A2
S113216080EE90E10E94550204C081E090E08AA3D1
S11321709BA3809102018B83CE010E94DA07EC01BC
S113218006C02093B00188E495E10E9455028FB700
S1132190F894282F3327209719F0F801C483D583A6
S11321A0F8011282138211828091B7028F5F8170CD
S11321B08093B7022FBFDF91CF911F910F910895A4
S11321C020918D0231E08FB7F8949091CE0291FD69
S11321D006C092609093CE0220938B0201C030E03F
S11321E08FBF313011F40E94FF0B089590E020E07E
S11321F030E0E091AA01F091AB01E20FF31F8FEF01
S113220080839F5F2F5F3F4F983098F3EAEBF1E0B4
S11322109F01295F3F4F8FEF81932E173F07DCF714
S113222085E191E10E9455020895DB981D9894E898
S113223080E02FB7F894422F552767E72BB3262366
S11322402BBB97FDDF9ADB9ACE9980682BBB96FD5A
S1132250DF9ADB9ACE9980642BBB95FDDF9ADB9ADB
S1132260CE9980622BBB94FDDF9ADB9ACE99806174
S11322702BBB93FDDF9ADB9ACE9988602BBB92FD32
S1132280DF9ADB9ACE9984602BBB91FDDF9ADB9AAF
S1132290CE9982602BBB90FDDF9ADB9ACE99816048
S11322A04FBF70E08FB7F894282F33279BB3962342
S11322B09BBB872F77FDDF9ADB9ACE9980689BBB07
S11322C076FDDF9ADB9ACE9980649BBB75FDDF9A1D
S11322D0DB9ACE9980629BBB74FDDF9ADB9ACE9920
S11322E080619BBB73FDDF9ADB9ACE9988609BBBB0
S11322F072FDDF9ADB9ACE9984609BBB71FDDF9AF5
S1132300DB9ACE9982609BBB70FDDF9ADB9ACE99F3
S113231081602FBF8FB7F894282F33279BB3962360
S11323209BBB872F77FDDF9ADB9ACE9980689BBB96
S113233076FDDF9ADB9ACE9980649BBB75FDDF9AAC
S1132340DB9ACE9980629BBB74FDDF9ADB9ACE99AF
S113235080619BBB73FDDF9ADB9ACE9988609BBB3F
S113236072FDDF9ADB9ACE9984609BBB71FDDF9A84
S1132370DB9ACE9982609BBB70FDDF9ADB9ACE9983
S113238081602FBF8FB7F894282F33279BB39623F0
S11323909BBB872F77FDDF9ADB9ACE9980689BBB26
S11323A076FDDF9ADB9ACE9980649BBB75FDDF9A3C
S11323B0DB9ACE9980629BBB74FDDF9ADB9ACE993F
S11323C080619BBB73FDDF9ADB9ACE9988609BBBCF
S11323D072FDDF9ADB9ACE9984609BBB71FDDF9A14
S11323E0DB9ACE9982609BBB70FDDF9ADB9ACE9913
S11323F081602FBF91E08FB7F894482F55272BB3F6
S113240026232BBB872F97FDDF9ADB9ACE99806812
S11324102BBB96FDDF9ADB9ACE9980642BBB95FD8E
S1132420DF9ADB9ACE9980622BBB94FDDF9ADB9A0C
S1132430CE9980612BBB93FDDF9ADB9ACE9988609D
S11324402BBB92FDDF9ADB9ACE9984602BBB91FD66
S1132450DF9ADB9ACE9982602BBB90FDDF9ADB9AE0
S1132460CE9981604FBF9FE88FB7F894482F5527C6
S11324702BB326232BBB872F97FDDF9ADB9ACE99AC
S113248080682BBB96FDDF9ADB9ACE9980642BBBC8
S113249095FDDF9ADB9ACE9980622BBB94FDDF9A7F
S11324A0DB9ACE9980612BBB93FDDF9ADB9ACE99A0
S11324B088602BBB92FDDF9ADB9ACE9984602BBB9C
S11324C091FDDF9ADB9ACE9982602BBB90FDDF9A57
S11324D0DB9ACE9981604FBF99E08FB7F894482F6B
S11324E055272BB326232BBB872F97FDDF9ADB9A27
S11324F0CE9980682BBB96FDDF9ADB9ACE998064D7
S11325002BBB95FDDF9ADB9ACE9980622BBB94FDA1
S1132510DF9ADB9ACE9980612BBB93FDDF9ADB9A1D
S1132520CE9988602BBB92FDDF9ADB9ACE998460AA
S11325302BBB91FDDF9ADB9ACE9982602BBB90FD79
S1132540DF9ADB9ACE9981604FBF1D9A84E690E0B2
S11325500197F1F7DB981D9894ED8FB7F894482F05
S113256055272BB326232BBB872F97FDDF9ADB9AA6
S1132570CE9980682BBB96FDDF9ADB9ACE99806456
S11325802BBB95FDDF9ADB9ACE9980622BBB94FD21
S1132590DF9ADB9ACE9980612BBB93FDDF9ADB9A9D
S11325A0CE9988602BBB92FDDF9ADB9ACE9984602A
S11325B02BBB91FDDF9ADB9ACE9982602BBB90FDF9
S11325C0DF9ADB9ACE9981604FBF8FB7F894282F9A
S11325D033279BB396239BBB872F77FDDF9ADB9A28
S11325E0CE9980689BBB76FDDF9ADB9ACE99806496
S11325F09BBB75FDDF9ADB9ACE9980629BBB74FD11
S1132600DF9ADB9ACE9980619BBB73FDDF9ADB9ADC
S1132610CE9988609BBB72FDDF9ADB9ACE99846069
S11326209BBB71FDDF9ADB9ACE9982609BBB70FDE8
S1132630DF9ADB9ACE9981602FBF8FB7F894282F49
S113264033279BB396239BBB872F77FDDF9ADB9AB7
S1132650CE9980689BBB76FDDF9ADB9ACE99806425
S11326609BBB75FDDF9ADB9ACE9980629BBB74FDA0
S1132670DF9ADB9ACE9980619BBB73FDDF9ADB9A6C
S1132680CE9988609BBB72FDDF9ADB9ACE998460F9
S11326909BBB71FDDF9ADB9ACE9982609BBB70FD78
S11326A0DF9ADB9ACE9981602FBF8FB7F894282FD9
S11326B033279BB396239BBB872F77FDDF9ADB9A47
S11326C0CE9980689BBB76FDDF9ADB9ACE998064B5
S11326D09BBB75FDDF9ADB9ACE9980629BBB74FD30
S11326E0DF9ADB9ACE9980619BBB73FDDF9ADB9AFC
S11326F0CE9988609BBB72FDDF9ADB9ACE99846089
S11327009BBB71FDDF9ADB9ACE9982609BBB70FD07
S1132710DF9ADB9ACE9981602FBF8FB7F894282F68
S113272033279BB396239BBB872F77FDDF9ADB9AD6
S1132730CE9980689BBB76FDDF9ADB9ACE99806444
S11327409BBB75FDDF9ADB9ACE9980629BBB74FDBF
S1132750DF9ADB9ACE9980619BBB73FDDF9ADB9A8B
S1132760CE9988609BBB72FDDF9ADB9ACE99846018
S11327709BBB71FDDF9ADB9ACE9982609BBB70FD97
S1132780DF9ADB9ACE9981602FBF8FB7F894282FF8
S113279033279BB396239BBB872F77FDDF9ADB9A66
S11327A0CE9980689BBB76FDDF9ADB9ACE998064D4
S11327B09BBB75FDDF9ADB9ACE9980629BBB74FD4F
S11327C0DF9ADB9ACE9980619BBB73FDDF9ADB9A1B
S11327D0CE9988609BBB72FDDF9ADB9ACE998460A8
S11327E09BBB71FDDF9ADB9ACE9982609BBB70FD27
S11327F0DF9ADB9ACE9981602FBF8093C2018FB795
S1132800F894282F33279BB396239BBB872F77FD00
S1132810DF9ADB9ACE9980689BBB76FDDF9ADB9AC0
S1132820CE9980649BBB75FDDF9ADB9ACE9980625A
S11328309BBB74FDDF9ADB9ACE9980619BBB73FDD1
S1132840DF9ADB9ACE9988609BBB72FDDF9ADB9A94
S1132850CE9984609BBB71FDDF9ADB9ACE9982602E
S11328609BBB70FDDF9ADB9ACE9981602FBF80936A
S1132870C3018FB7F894282F33279BB396239BBBB0
S1132880872F77FDDF9ADB9ACE9980689BBB76FD14
S1132890DF9ADB9ACE9980649BBB75FDDF9ADB9A45
S11328A0CE9980629BBB74FDDF9ADB9ACE998061DE
S11328B09BBB73FDDF9ADB9ACE9988609BBB72FD4C
S11328C0DF9ADB9ACE9984609BBB71FDDF9ADB9A19
S11328D0CE9982609BBB70FDDF9ADB9ACE998160B2
S11328E02FBF8093C4011D9A20E034E040E050E003
S11328F0672F872F0E94430708951F93CF93DF9379
S11329009091EF01992319F483E090E015C0809130
S1132910A701823019F48FEF8093A7018091A7015A
S11329208F5F8093A70191509093EF01E82FFF27C9
S1132930E455FE4F80819927833008F0A5C099277C
S113294081309105D1F0823091051CF4892B21F05E
S11329509BC00297F9F098C08FB7F894C82FDD2771
S113296080917A02882339F481E080937A0285E5A4
S113297095E10E945502CFBF87C080915C0290917F
S11329805D029093BB028093BA0210925D02109292
S11329905C027AC0E0918C02EE2309F475C08FB713
S11329A0F89499272091B1011091AF018FBF33277B
S11329B02230310521F02630310591F15DC08E2F92
S11329C09927880F991FFC01EF55FF4F2491332756
S11329D0D22FCC278E559F4FFC0184919927C82B69
S11329E0D92B112309F048C08FB7F894282F332727
S11329F086E08093B1012FBFCE01AA27BB279C019B
S1132A00AD0161E082E00E944307612F8BE00E94E8
S1132A10D1066FE3812F0E94D1060E94BA0B34C005
S1132A20FF27E155FF4F8491C82FDD278FB7F89416
S1132A30992712E01093B1018FBF6BE380E00E94ED
S1132A40D10680ED97E00197F1F769E380E00E94F9
S1132A50D10688EC90E00197F1F7BB98BA980E94F0
S1132A60C20780EC8DB9B8980E94B007CE01AA279E
S1132A70BB279C01AD0104C020E230E040E050E0FF
S1132A8061E082E00E944307DF91CF911F91089596
S1132A908FB7F894282F33278091CE0288608093D3
S1132AA0CE022FBF0E94FF0B0895EF92FF921F9357
S1132AB0CF938091CA0191E089278093CA0188232A
S1132AC021F01EE7E12EF12C03C0CFEFEC2EFC2EFB
S1132AD08091D1028F5F8093D1029FB7F894877061
S1132AE08093A30281FF02C0D99801C0D99A809132
S1132AF0A30282FF02C0D89801C0D89A80FF02C006
S1132B00DA9801C0DA9A9FBFC091C002CC2329F59C
S1132B1011E01093C00282EB95E10E9455028823D4
S1132B2019F4C093C00219C085EB91E09093ED01B4
S1132B308093EC0181E18093B901F092B601E092B7
S1132B40B5018AE08093B701809102018093B801B6
S1132B50812F8E5F8C5F8B32E8F3CF911F91FF90B2
S1132B60EF9008951F93CF93E091EC01F091ED0164
S1132B70808191818E379105C1F461E08FB7F8941B
S1132B809091CE0292FD08C094609093CE02F0938F
S1132B90A601E093A50101C060E08FBF613009F098
S1132BA07EC00E94FF0B682F7AC011E08FB7F894A3
S1132BB0C82F8091A901882311F010E018C0109348
S1132BC0A901F093A502E093A402848199270596B4
S1132BD09093EB018093EA010E94970B8F7790709A
S1132BE0849690938702809386021093AF01CFBF9F
S1132BF0112309F453C08FB7F89499272091B10198
S1132C008FBF263009F04AC04091C1025091C202E0
S1132C106091C3027091C40242FF17C08FB7F89449
S1132C20282F3327DB01CA018B7F8093C102909345
S1132C30C202A093C302B093C4022FBF0097A105A0
S1132C40B10519F481E0809383026BE380E00E9474
S1132C50D10680ED97E00197F1F769E380E00E94E7
S1132C60D10688EC90E00197F1F70E94C207BB9867
S1132C70BA9880EC8DB9B8980E94B00720E230E091
S1132C8040E050E061E082E00E9443078FB7F8948F
S1132C90282F332782E08093B1012FBF612F662351
S1132CA031F48091EC019091ED010E94880BCF9159
S1132CB01F910895629FD001739FF001829FE00DE0
S1132CC0F11D649FE00DF11D929FF00D839FF00DA7
S1132CD0749FF00D659FF00D9927729FB00DE11D53
S1132CE0F91F639FB00DE11DF91FBD01CF01112430
S1132CF00895A1E21A2EAA1BBB1BFD010DC0AA1F39
S1132D00BB1FEE1FFF1FA217B307E407F50720F050
S1132D10A21BB30BE40BF50B661F771F881F991FCB
S1132D201A9469F760957095809590959B01AC0114
S1092D30BD01CF0108956E
S1132D36010033008025009224200000201C00009E
S1132D46001900008016005D74140000C01200C54E
S1132D564E110049121000BD04880552061C07E6F0
S1132D6607B0087B09450A0F0BAA01F10138028056
S10F2D7602C7020E0355039C03E3030193
S9030000FC
